:1000000012C0189518951895189518951895189563
:100010001895189518951895189518951895189578
:100020001895189518958FE58DBFC8E3E0E24E2E20
:1000300084E08EBFD4E0F4E05F2EA89584B7082E4C
:10004000877F84BF88E1992781BD91BDEEEFF3E002
:10005000A0E6B0E088278D933197E9F770D8662441
:100060008CE0B5D852D883E886B980E487B9A49AE1
:10007000A59AB998BA98BB98C19AC29AC39AAAEAA3
:10008000B0E0E2E0F0E094E0B4DCAEEAB0E0E6E05C
:10009000F0E094E0AEDCE0E0F0E0A6E9B0E0A6DC61
:1000A000E1E0F0E0A7E9B0E0A1DCEBE0F0E0A6EBF6
:1000B000B0E09CDCECE0F0E0A7EBB0E097DCEDE03A
:1000C000F0E0A8EBB0E092DCEEE0F0E0A9EBB0E00D
:1000D0008DDC0091B700073110F009F001C00CC0B1
:1000E00080E08093B60080E08093B70080E080934A
:1000F000B80080E08093B900E0E1F1E080E467D8E7
:1001000058E0C895802D5DD831965A95D1F704C036
:10011000181C1E1F1F1E1C18E0E3F1E088E457D8CE
:1001200058E0C895802D4DD831965A95D1F704C026
:100130000E0A0A20040C0404E0E5F1E080E547D84B
:1001400058E0C895802D3DD831965A95D1F704C016
:100150000E0A0A200E02040EE0E7F1E088E637D826
:1001600058E0C895802D2DD831965A95D1F704C006
:100170002020202020202020E0E9F1E080E727D87F
:1001800058E0C895802D1DD831965A95D1F704C0F6
:1001900002050220202020208FE711E0C5D7E4E2ED
:1001A000FBE1ADD78FEB11E0BFD7EEE2FBE1A7D7C4
:1001B000379AABD782E0E0E35BDBA0E7B0E00D93DA
:1001C0001C9382E0E0E3DFDAA2E7B0E0E5EEF0E0E6
:1001D00098E0F0DB82E0E0E3DBDAAAE7B0E0E5EE0E
:1001E000F0E098E0E7DB82E0E0E3D2DAA2E8B0E01A
:1001F000E5EEF0E098E0DEDB62FA0EF0F4CFA0E787
:10020000B0E00D911C91033050E0150708F00CC0D0
:100210008FE711E089D7E8E3FBE171D78FEB11E0BD
:1002200083D7E2E4FBE16BD788EC90E014D8A0E739
:10023000B0E00D911C91033050E0150709F0BACFE2
:1002400087E0E2E7F0E0FFDB402F00917900041740
:1002500009F011C05AD78FE711E066D7E8E3FBE158
:100260004ED78FEB11E060D7ECE4FBE148D7E1E03B
:10027000F0E05CD70FC08FE711E056D7E8E3FBE171
:100280003ED78FEB11E050D7E6E5FBE138D7E1E050
:10029000F0E04CD787E0EAE7F0E0D5DB402F0091B3
:1002A0008100041709F011C030D78FE711E03CD767
:1002B000E8E3FBE124D78FEB11E036D7E0E6FBE182
:1002C0001ED7E1E0F0E032D70FC08FE711E02CD766
:1002D000E8E3FBE114D78FEB11E026D7EAE6FBE178
:1002E0000ED7E1E0F0E022D787E0E2E8F0E0ABDB18
:1002F000402F00918900041709F011C006D78FE73D
:1003000011E012D7E8E3FBE1FAD68FEB11E00CD74E
:10031000E4E7FBE1F4D6E1E0F0E008D70FC08FE7B7
:1003200011E002D7E8E3FBE1EAD68FEB11E0FCD65F
:10033000EEE7FBE1E4D6E1E0F0E0F8D6E6D68FE7C1
:1003400011E0F2D6E8E8FBE1DAD687E290E0AEE62B
:10035000B0E08D939C9384EF91E07DD7AEE6B0E062
:10036000B8D6AEE6B0E00D911C91083250E015070A
:1003700009F0B9C081E08093D40026D282E0809356
:10038000D40022D283E08093D4001ED2EDD080E04E
:1003900090E0AEE6B0E08D939C938091D80080937E
:1003A000A4008091D7008093A50051D6E6EAF0E042
:1003B000A2EBB0E0FEDAE2EBF0E0ABD7EEEAF0E081
:1003C000ADD758D781E008F480E08F93E2EBF0E0FE
:1003D000A0D7EAEAF0E0A2D74DD781E008F080E0AC
:1003E0009F918923882309F40CC0AC98AD9880E0D4
:1003F0008093CF0080E08093D00080E08093D10094
:1004000072C081E08093D1004091960000919000ED
:10041000041781E008F480E08F930091D30000304E
:1004200081E009F080E09F918923882309F404C0CA
:10043000AC9880E08093CF004091960000919100AD
:10044000041781E008F480E08F930091D30000301E
:1004500081E009F080E09F918923882309F404C09A
:10046000AD9880E08093D00040919700009190007B
:10047000041781E010F009F080E08F930091D30021
:10048000003081E009F080E09F918923882309F4FE
:1004900004C0AC9A81E08093CF0040919700009116
:1004A0009100041781E010F009F080E08F93009133
:1004B000D300003081E009F080E09F9189238823F8
:1004C00009F404C0AD9A81E08093D0000091D3007C
:1004D000013009F008C0AC98AD9880E08093CF005F
:1004E00080E08093D0000091D100013009F021C05C
:1004F0000091CF00013009F006C08FEB17E014D651
:1005000081E05FD605C08FEB17E00ED685E059D6A7
:100510000091D000013009F006C08FEB18E004D63E
:1005200082E04FD605C08FEB18E0FED585E049D6B6
:1005300006C08FEB17E0F8D5E2E9FBE1E0D515D274
:100540000091CE00033009F001C096C20091CE00A8
:10055000023009F001C0A4D00091CE00013009F0B2
:1005600001C0DBD058D0F7CE83DA10ED97DA10E077
:1005700095DA7EDA11ED92DAB0DAA6EDB0E01C93EE
:10058000ACDAA7EDB0E01C93A8DAA8EDB0E01C93BC
:10059000A4DAA9EDB0E01C93A0DAAAEDB0E01C93B8
:1005A0009CDAABEDB0E01C9396DAACEDB0E01C93B6
:1005B0006CDAA6EDB0E09C913BD6A6EDB0E08C9352
:1005C000A7EDB0E09C9134D6A7EDB0E08C93A8EDF8
:1005D000B0E09C912DD6A8EDB0E08C93A9EDB0E0F1
:1005E0009C9126D6A9EDB0E08C93AAEDB0E09C9149
:1005F0001FD6AAEDB0E08C93ABEDB0E09C9118D67D
:10060000ABEDB0E08C93ACEDB0E09C9111D6ACEDCD
:10061000B0E08C9308950091D300003009F033C00E
:100620008FE712E081D5AAE6B0E063D586E0C9D5B0
:10063000E6E9FBE164D58FEB11E076D5A8E0B4E004
:10064000E8EDF0E067D953D5EAE9FBE158D5009130
:10065000D7000A3008F00DC0ECE9FBE150D5A8E066
:10066000B4E0E7EDF0E056D942D5EEE9FBE147D53D
:1006700009C0A8E0B4E0E7EDF0E04CD938D5EEE9E8
:10068000FBE13DD50CC08FE711E04ED5E8E3FBE17F
:1006900036D58FEB11E048D5E2E4FBE130D5089583
:1006A00034D50091D300003009F023C08FE713E068
:1006B0003BD5E0EAFBE123D58FE711E035D5E6EA4B
:1006C000FBE11DD5A2E6B0E014D586E07AD5EAEAD2
:1006D000FBE115D58FEB11E027D5ECEAFBE10FD557
:1006E000A6E6B0E006D586E06CD5EAEAFBE107D5E0
:1006F0000CC08FE711E018D5E8E3FBE100D58FEBE4
:1007000011E012D5E2E4FBE1FAD4E3E0F0E00ED52B
:10071000FCD480E08093CE000895F7D48FE711E0F9
:1007200003D5E0EBFBE1EBD4A8E0B4E0E7EBF0E0CD
:10073000F1D8DDD4EAE9FBE1E2D40091B6000A3059
:1007400008F00AC0ECE9FBE1DAD4A8E0B4E0E6EB9B
:10075000F0E0E0D8CCD409C0A8E0B4E0E6EBF0E0EB
:10076000D9D8C5D4EEE9FBE1CAD48FEB11E0DCD4D3
:10077000E4EBFBE1C4D4A8E0B4E0E9EBF0E0CAD8D4
:10078000B6D4EAE9FBE1BBD40091B8000A3008F026
:100790000AC0ECE9FBE1B3D4A8E0B4E0E8EBF0E098
:1007A000B9D8A5D409C0A8E0B4E0E8EBF0E0B2D82D
:1007B0009ED4EEE9FBE1A3D4E3E0F0E0B7D4A5D406
:1007C00080E08093CE00089582E0E0E33AD75CECCD
:1007D00082E0E0E358D754E482E0E0E354D780E2DB
:1007E00093E039D50091D400013009F005C082E0D2
:1007F000E0E3A2E7B0E04FD80091D400023009F066
:1008000005C082E0E0E3AAE7B0E045D80091D4005B
:10081000033009F005C082E0E0E3A2E8B0E03BD895
:1008200062FA0EF49EC05EEB82E0E0E32CD7BB27B9
:10083000A6E182E0E0E321E02A934DD7AAE8B0E008
:100840005C93BB27A6E182E0E0E321E02A9343D753
:10085000ABE8B0E05C9300918B00083F08F414C053
:100860000FEF40918A00041BAAE8B0E00C930FEF51
:1008700040918B00041BABE8B0E00C93ACE8B0E017
:10088000E8EBFBE138D505C0ACE8B0E0EAEBFBE112
:1008900032D500918A0040E1B3D8AEE8B0E00C93C5
:1008A00000918B0040E1049FAFE8B0E00C92009112
:1008B0008E0040918F00040FAEE8B0E00C93ACE8DE
:1008C000B0E0E8EBFBE1ACD809F005C0AEE8B0E081
:1008D0008C918F5F8C9300918E00003009F005C0E1
:1008E000ACE8B0E0EEE9FBE106D580E08093D30010
:1008F0000091D400013009F00FC0ECE8F0E0A2E66E
:10090000B0E052D8A2E6B0E0EBD3EEE8F0E002D8D7
:1009100080918E00809390000091D400023009F005
:100920000FC0ECE8F0E0A6E6B0E03ED8A6E6B0E006
:10093000D7D3EEE8F0E0EED780918E00809391005F
:100940000091D400033009F00BC0ECE8F0E0AAE617
:10095000B0E02AD8AAE6B0E0C3D3EEE8F0E0DAD7F8
:1009600003C081E08093D300089580E08093CE009F
:1009700007B1007F036007B9C3D4A0E6B0E08D9350
:100980009C93E0E1FBE16FD5E0E6F0E0D190E08000
:100990008FEFE7FE8827F82E082FCDD40AD5EDE09B
:1009A000F0E0ADEDB0E005D8EDEDF0E0B2D4E4E17B
:1009B000FBE159D55FD409F003C080E08093D200F9
:1009C0000091D200003009F053C0EDEDF0E0A1D469
:1009D000E8E1FBE148D54ED480E010F009F081E079
:1009E0008F93EDEDF0E095D4ECE1FBE13CD542D402
:1009F00081E008F080E09F918923882309F406C0F4
:100A000081E08093CE0081E08093D200EDEDF0E0B4
:100A100080D4ECE1FBE127D52DD480E010F009F083
:100A200081E08F93EDEDF0E074D4E0E2FBE11BD5C3
:100A300021D481E008F080E09F918923882309F484
:100A400006C082E08093CE0082E08093D200EDED7C
:100A5000F0E05FD4E0E2FBE106D50CD410F009F041
:100A600001C006C083E08093CE0083E08093D20073
:100A700082E390E0F0D3089581E08093CD0045D3E8
:100A800074DF0091CE00013009F001C05BC000911D
:100A9000CE00023009F001C045C00091CE00033005
:100AA00009F001C05DC00091CD00013009F005C022
:100AB000ACEBB0E0ECEBFBE11ED40091CD000230DA
:100AC00009F005C0ACEBB0E0E6ECFBE114D400911A
:100AD000CD00033009F005C0ACEBB0E0E0EDFBE188
:100AE0000AD40091CD00043009F005C0ACEBB0E0B1
:100AF000EAEDFBE100D40091CD00053009F005C01E
:100B0000ACEBB0E0E4EEFBE1F6D38FE711E00CD301
:100B1000EEEEFBE1F4D28FEB11E006D3ACEBB0E0EC
:100B2000E8D2AECFADECB0E08C918F5F8C930091AA
:100B3000CD00053010F009F001C003C085E08093BE
:100B4000CD009DCF8091CD0081508093CD0000914C
:100B5000CD00013008F003C081E08093CD008FCF3D
:100B60000091CD00013009F001C019C00091CD0005
:100B7000023009F001C0BEC00091CD00033009F081
:100B800001C025C10091CD00043009F001C08CC125
:100B90000091CD00053009F001C0F4C1E1CFE4DCE3
:100BA0008091D8008093BA008091D7008093BB00D9
:100BB000ACD28FE711E0B8D2ECEBFBE1A0D28FEB27
:100BC00011E0B2D2E8EFFBE19AD2A8E0B4E0E8EDA0
:100BD000F0E0A0D68CD2EAE9FBE191D20091D700F7
:100BE0000A3008F00AC0ECE9FBE189D2A8E0B4E0E1
:100BF000E7EDF0E08FD67BD206C0A8E0B4E0E7EDE9
:100C0000F0E088D674D2B1DE0091CE00013009F058
:100C100001C00DC00091CE00023009F001C017C024
:100C20000091CE00033009F001C021C0C8CFA8ED6B
:100C3000B0E08C918F5F8C930091D800073110F059
:100C400009F001C003C080E08093D800B1CFA7EDC8
:100C5000B0E08C918F5F8C930091D7000B3310F034
:100C600009F001C003C080E08093D700A1CF40917C
:100C7000D8000091BA00041781E009F080E08F935A
:100C80004091D7000091BB00041781E009F080E09B
:100C90009F918923882309F402C0F1CE2AC081E004
:100CA0008093D600A6EDB0E08C91BCD2A6EDB0E06A
:100CB0008C93A7EDB0E08C91B5D2A7EDB0E08C930A
:100CC000A8EDB0E08C91AED2A8EDB0E08C93D0D678
:100CD00010EDE4D610E0E2D6A6EDB0E01C91DED631
:100CE000A7EDB0E01C91DAD6A8EDB0E01C91D6D605
:100CF000CCD6C5CE0AD28FE711E016D2E6ECFBE1E6
:100D0000FED18091B7008093A4008091B6008093BB
:100D1000A5009DD1E6EAF0E0AAEAB0E04AD68FEB62
:100D200011E002D2E8EFFBE1EAD1A8E0B4E0E7EBA2
:100D3000F0E0F0D5DCD1EAE9FBE1E1D10091B600C9
:100D40000A3008F00AC0ECE9FBE1D9D1A8E0B4E030
:100D5000E6EBF0E0DFD5CBD106C0A8E0B4E0E6EBEF
:100D6000F0E0D8D5C4D101DE0091CE00013009F009
:100D700001C00DC00091CE00023009F001C017C0C3
:100D80000091CE00033009F001C079CEC8CFA7EBA7
:100D9000B0E08C918F5F8C930091B700073110F019
:100DA00009F001C003C080E08093B700A3CFA6EB99
:100DB000B0E08C918F5F8C930091B6000B3310F0F4
:100DC00009F001C003C080E08093B60093CF9DD1AD
:100DD0008FE711E0A9D1E0EDFBE191D18091B9005D
:100DE0008093A4008091B8008093A50030D1E6EAFA
:100DF000F0E0AEEAB0E0DDD58FEB11E095D1E8EFA1
:100E0000FBE17DD1A8E0B4E0E9EBF0E083D56FD160
:100E1000EAE9FBE174D10091B8000A3008F00AC099
:100E2000ECE9FBE16CD1A8E0B4E0E8EBF0E072D5CE
:100E30005ED106C0A8E0B4E0E8EBF0E06BD557D196
:100E400094DD0091CE00013009F001C00DC0009189
:100E5000CE00023009F001C017C00091CE0003306F
:100E600009F001C00CCEC8CFA9EBB0E08C918F5F28
:100E70008C930091B900073110F009F001C003C054
:100E800080E08093B900A3CFA8EBB0E08C918F5F96
:100E90008C930091B8000B3310F009F001C003C02F
:100EA00080E08093B80093CFB8D0ACD08FE711E04A
:100EB0003BD180E086D159DD0091CE00023009F0AF
:100EC00001C00DC00091CE00013009F001C017C073
:100ED0000091CE00033009F001C01DC0ECCFA6E99F
:100EE000B0E08C918F5F8C9300919600033610F0E8
:100EF00009F001C003C083E680939600D5CF00912E
:100F00009600003009F001C0CFCF8091960081504B
:100F100080939600C9CF81D075D08FEB11E004D1BA
:100F200080E04FD122DD0091CE00023009F001C0F7
:100F30000DC00091CE00013009F001C017C0009132
:100F4000CE00033009F001C09ACDECCFA7E9B0E0A4
:100F50008C918F5F8C9300919700033610F009F00D
:100F600001C003C083E680939700D5CF009197001E
:100F7000003009F001C0CFCF80919700815080935D
:100F80009700C9CFC2D08FE711E0CED0ECEFFBE1E4
:100F9000B6D0E1E0F0E0CAD0E2E0F0E0AAEAB0E0EA
:100FA00094E07BE715D5E6E0F0E0AEEAB0E094E04F
:100FB0007BE70ED5EBE0F0E0A6EBB0E07BE705D5F4
:100FC000ECE0F0E0A7EBB0E07BE7FFD4EDE0F0E091
:100FD000A8EBB0E07BE7F9D4EEE0F0E0A9EBB0E0FD
:100FE0007BE7F3D4E0E0F0E0A6E9B0E07BE7EDD406
:100FF000E1E0F0E0A7E9B0E07BE7E7D480E08093B0
:10100000CE00A3C98FE711E08FD085E0DAD08FEB57
:1010100011E08AD085E0D5D0089577D08FE711E030
:1010200083D0E6E0FCE16BD0A8E0B4E0E6E9F0E0D4
:1010300071D45DD08FEB11E077D0EEE0FCE15FD0B2
:10104000A8E0B4E0E7E9F0E065D451D00895A8E95C
:10105000B0E0E4EAF0E05ED4ABE9B0E0E5EAF0E06D
:1010600059D40091A5000A3008F017C084E03DD1A2
:10107000EBE9F0E0A881B98197D4ABE9B0E0ECE905
:10108000FBE139D1E881F981ABE9B0E029D08CD41A
:1010900084E0481A80E0580A2296E8E9F0E0AEE9D8
:1010A000B0E082D4AEE9B0E01BD0E6E1FCE123D1B0
:1010B000EBE9F0E0AEE9B0E013D076D4AEE9B0E011
:1010C000DBD1EDE0F0E0A6EAB0E073D40895F89447
:1010D000FFCFED91FC91EF5FFF4FFC93EE930895EE
:1010E0008F938D918823E9F711978F910895A8E048
:1010F000B4E08D91882311F064D0FBCF0895AFD177
:10110000802D11F05ED0FBCF089581E060D014D027
:1011100080E85DC08FE7213039F08FEB223021F07D
:101120008FE8233009F08FEC810F51C088EE93E0F7
:1011300092D03197D9F7089583E099278CC08AEF30
:1011400090E089D0B89A8F9A8E9A8D9ABF9ABE9A5B
:10115000C69885E090E07FD0C798C0989798969AF7
:10116000959AC79AEF93FF93E5E1F0E068D0FF917D
:10117000EF91C7986DD0C79AEF93FF93E5E1F0E048
:101180005ED0FF91EF91C79863D0C79AEF93FF931A
:10119000E5E1F0E054D0FF91EF91C79859D09598D0
:1011A000C79AEF93FF93E5E1F0E049D0FF91EF910B
:1011B000C7984ED088E20BD08EE009D086E007D0E9
:1011C0000895C69A829505D004D042D00895C69855
:1011D000F9CF859510F4959A01C09598859510F4EE
:1011E000969A01C09698859510F4979A01C09798A1
:1011F000859510F4C09A01C0C098C79AEF93FF93E9
:10120000E5E1F0E01CD0FF91EF91C7980895982F89
:1012100082958F70805D8D939F70905D9D938827E0
:101220008C9308954AE0082FEBD30295802B089504
:10123000892F8F70905110F0865FFCCF0895319701
:10124000F1F70895689462F80895E89462F80895B3
:1012500081E090E000C0EF93FF93EE27E82BE92BAD
:1012600031F0EAEFF0E03197F1F70197D1F7FF9114
:10127000EF9108958F939F93D216E306F4060FB66D
:1012800080E890E8802795270FBE89070FB6892B45
:1012900087FD02C091E009260FBE9F918F910895AE
:1012A000B7FE089590E8B91611F4D0FE08959FEFA7
:1012B000D91AE90AF90A09F403950895652F90E807
:1012C000440F551F5927990F47956078102F90E8C4
:1012D000FF0C001F0927990FF79410780038089524
:1012E0005A924A92480E591E08955A924A92480EAE
:1012F0008827581E0895B3D00D920020E1F7089575
:10130000369A3699FECF369A3699FECF84B195B18A
:101310000895D190E190F19001910895219131913A
:10132000419151910895FF0C90E89027110F9795E6
:10133000F794092F0895102FBD2CDE2CEF2CF02EE2
:1013400011234AF4B094D094E094F0949FEFB91A2A
:10135000D90AE90AF90A0EE1FF2039F4FE2CED2C36
:10136000DB2CBB240850C2F758C032F00A95BB0CE6
:10137000DD1CEE1CFF1CF9CF93DFD5CF502F2D2D98
:101380003E2D4F2D612F08952DEC3CEC4CEC5DE390
:1013900066270FC0BEDFF2DFDD24EE2490E8F92ED1
:1013A0000FE307C0BBDF05C02227332740E251E42B
:1013B0006627552351F1002381F180DF71F1162753
:1013C000005850580894050B18F407FD03C025C0B9
:1013D00007FD23C0469537952795F694E794D79453
:1013E00022D0FF202AF0DD0CEE1CFF1C015073F010
:1013F0009D2D969548F0DD203AF4EE202AF491E0F8
:10140000D90E9927E91EF91E8ECF07C09FE7092F35
:10141000F92A9FEFD92EE92E0895DD24EE24FF242A
:101420000027112708959F929924AA24BB2488E1BC
:10143000D216E306F40628F0D21AE30AF40A089456
:1014400001C08894991CAA1CBB1CDD0CEE1CFF1C5F
:101450008A9571F7D92CEA2CFB2C9F900895C8959A
:10146000319600200895FBDF202DF9DF302DF7DFC6
:10147000402DF5DF502D0895E8DEE89488278A9303
:101480008A93CBDF11278D918032E9F31197BAD07F
:1014900090F08D3229F4109511968C91B3D058F0BC
:1014A0008E3229F411968C91ADD008F445C0229665
:1014B000C9DE81E008958C91A5D0D8F547D011966A
:1014C000D0F703958D919ED0E0F38E3229F48C9164
:1014D00099D010F41196FBCF853419F0853609F0B8
:1014E00055C011968C918ED060F08D3219F08B32F0
:1014F00021F0DDCF08800094088211968C9182D073
:10150000B0F68053898311968C917CD058F49981E0
:10151000990F990F0980900D990F8053890F898336
:10152000873228F68981988199230AF48195080FDA
:101530002DC08E3289F611968C9164D068F606D053
:1015400018F011960A95F8CF1196C1CF4F2D3E2D68
:101550002D2DDD0CEE1CFF1CA8F0DD0CEE1CFF1C7D
:1015600088F0D20EE31EF41E68F0DD0CEE1CFF1CAA
:1015700048F0805309F06894D80E8827E81EF81EBA
:1015800008F00895F42EE32ED22E089534D019F1E8
:1015900016F5098308E921D00695882787959F2DA0
:1015A0009F77980FF92E0150000F110F0795898131
:1015B000882379F01AF48195898306C0E5DE898154
:1015C0008A958983D9F705C0EFDE89818A95898359
:1015D000D9F72296089521DFFCCF0DD041F0FF20EE
:1015E00032F00A9531F0DD0CEE1CFF1CD2F7889426
:1015F00008950894089500240D280E280F28002A25
:1016000000200895803320F08A3310F40894089560
:101610008894089591E0882321F08894991F8A95F1
:10162000E9F7892F90950895883018F01196885021
:10163000FBCF08950181082B0183128119231283A6
:10164000089503DEFF27E6DFF5DFEF93FF93E4E77E
:10165000F0E0F5DDFF91EF91182B12830923018350
:10166000EF93FF93EEE0F0E0EADDFF91EF91108160
:10167000182309F0E7DDEF93FF93E3E6F0E0DFDD09
:10168000FF91EF910895C6DFFF2721E048E005C0F4
:10169000C1DFFF2729915D9148E0CCDF579510F419
:1016A000182B1283EF93FF93EAE0F0E0C8DDFF917F
:1016B000EF91182B128300000000000000000000D2
:1016C0000000000000000000000000004A9529F71B
:1016D0002A9509F708959EDFFF27299148E05527AD
:1016E000A9DF0923018300000000000000000000C2
:1016F0000000000000000000000088941081182302
:1017000009F008945795EF93FF93EAE0F0E097DD36
:10171000FF91EF914A9521F75D932A95F9F6089587
:1017200089DF0923018300000000000000000000A1
:1017300000000000000000000000E8941081182361
:1017400009F06894EF93FF93EAE0F0E078DDFF9111
:10175000EF9108956FDF16F4182B1283EF93FF9328
:10176000EAE0F0E06CDDFF91EF91182B12830000AE
:101770000000000000000000000000000000000069
:1017800000000000089533273093E4003093E10017
:1017900058DF0EF458C03091E10030FD54C0662788
:1017A0006093E30063956093E20021E050EF48E02E
:1017B00074DFB6DF31F9B4DF32F9632F667066305B
:1017C00009F441C0603019F031FB40D025C0609170
:1017D000E2007091E4006717B1F0C0F48F939F931B
:1017E000862F8A95A5EEB0E01FDF14DF7C91782369
:1017F0006894772329F4E8946091E2006093E30011
:101800009F918F9109C0689421D006C0E8941ED0A2
:101810006091E2006093E3009DDF6091E2006395D8
:101820006093E200613409F0C4CF6091E3006093FB
:10183000E4006623E89409F4689430F93093E100F9
:10184000E89462F80895689462F808958F939F93DE
:10185000A5EEB0E08091E2008A95E6DEDBDE7C91C9
:1018600016F4782B01C079237C939F918F91089572
:101870008F9389DF8F91A0E0B0E056F011968F939F
:10188000AF93BF9385DFBF91AF918F910EF0F6CFED
:101890000A2F1B2F0895AF93BF93EF93FF9338E068
:1018A000E5EEF0E00D9101933A95E1F7FF91EF91AC
:1018B00030E43093E40033273093E10069DF38E00F
:1018C000BF91AF91E5EEF0E00D914191041719F44D
:1018D0003A95D1F70895B6DC0895000F111F221F25
:1018E000331F089500951095209530950F5F1F4F79
:1018F0002F4F3F4F0895019110810EC0019111911A
:10190000219130810BC00191108117FF05C03FEF7D
:101910002FEF04C0008111272227332737FF03C090
:10192000E1DF8DE28D93CF93DF93CF92DF92EF9241
:10193000AA24BB24CC24DD24EE2440E2CAE0DD2727
:1019400055E093E38881890F87FD9F7083FD907F29
:10195000891B89935A95A9F7C0DFAA1CBB1CCC1C14
:10196000DD1CEE1C4A9551F7E894EFE0FF278291C9
:101970000ED0EB30E0F71EF068948A2D0CD088274B
:101980008D93EF90DF90CF90DF91CF910895982FB6
:10199000829501D0892F8F70805D26F0803309F405
:1019A000089568948D93089581918D938823E1F72C
:1019B000089594E081918D939A95E1F70895E199C6
:1019C000FECFEEBBFFBB3196089591E001C092E0DF
:1019D0007B3751F47FB7F894F2DF8D918DBBE29A9B
:1019E000E19A9A95C9F77FBF7727089591E001C0E2
:1019F00092E0E5DFE09A8DB38D939A95D1F7089543
:101A0000FF93881BF9E0001FFA9511F4FF910895E8
:101A1000881F841B18F4840F8894F5CF0894F3CFA3
:101A2000689401C0E894AF93BF938D9116F09191A3
:101A300002C015DD902D891718F011F48823A9F73D
:101A4000BF91AF91089500276CE8719198E00695D9
:101A5000779577FF18F477FD08F006279A95B9F780
:101A60008A9599F70895A998A898A198A09808959B
:101A7000A09AA19803D0A09801D0A19A00000000DC
:101A800000000000000000000895A09AA19AF6DF6F
:101A9000A098989BFECFF2DFA198F0CF0894111F79
:101AA00001C0110F69F0A09A18F40000A19802C0BB
:101AB000A19A00C0E3DFA098989BFECFDFDFF1CFB3
:101AC000A09AA198DBDFA098989BFECFE894999903
:101AD000689462F8D3CF089401C08894331F11E052
:101AE000A09AA198CBDFA098989BFECFC7DF8894DF
:101AF00099990894111FA0F7A09A379510F4A1980E
:101B000001C0A19ABBDFA098989BFECFB7DF0895D4
:101B10000000C842000000000000004000008040BB
:101B200000001041545020562E312E3100002D203F
:101B300032303131202D00002053656E736F7220DA
:101B40000000202045726F72202000004944313D82
:101B5000204F4B2000004944312045726F72000035
:101B60004944323D204F4B20000049443220457209
:101B70006F7200004944333D204F4B200000494420
:101B8000332045726F720000202D4C4F41442D20B0
:101B9000000020450000432000003A0030002000F3
:101BA000A86FBBC30000A8313A004300A8323A0036
:101BB0006F6E20006F6620002D002B00A963BF2EE2
:101BC000B3702DB8000042702E20B3BABB2E0000B7
:101BD00042702EB3C3BABB2E0000A963BF2EBF65EF
:101BE000BCBE00002042C3786FE3203E00003C20D2
:101BF0004D65BDC6203E00003E3E20002020436FC4
:101C000078702E200000542E6D61783D0000542E17
:081C10006D696E3D00002E001D
:00000001FF
